:100000000C943C020C9459020C9459020C94590221
:100010000C9459020C9459020C9459020C945902F4
:100020000C9459020C9459020C9423260C94F52636
:100030000C942A210C9459020C9459020C945902E4
:100040000C9459020C9459020C9459020C945902C4
:100050000C9459020C94B2210C9459020C9459023C
:100060000C9459020C9459020C9459020C945902A4
:100070000C9459020C9459020C9459020C94590294
:100080000C9459020C9459020C9459020C94590284
:100090000C9459020C9459020C9459020C94590274
:1000A0000C9459020C9459020C945902150515052B
:1000B00041054105A905C705DF06DF06D2056B0628
:1000C0007C067C0662278927812889278128D527F5
:1000D000F82781284F285E284C002C0028000000BB
:1000E0005000510052004F000158025803580000C0
:1000F000AC00AE00AB000000BE00AA00A900BD002D
:100100000100010001000000C45CC35CC55C00008C
:10011000680069006A006B00010001000100000036
:10012000B600B900B700000000004E004B00000010
:10013000010001000100000000047F3F1F64321431
:10014000643214783C1E1E140A0522232526282911
:100150002A2C2D2F3032333536383A3B3D3E404243
:10016000434547494A4C4E5051535557595A5C5E86
:100170006062646668696B6D6F71737577797B7D9A
:100180007F81838587898A8C8E90929496989A9C99
:100190009E9FA1A3A5A7A8AAACAEAFB1B3B4B6B8B1
:1001A000B9BBBCBEBFC1C2C3C5C6C7C9CACBCCCD13
:1001B000CED0D1D2D2D3D4D5D6D7D7D8D9D9DADAEE
:1001C000DBDBDBDCDCDCDCDCDDDDDDDDDCDCDCDC6E
:1001D000DCDBDBDBDADAD9D9D8D7D7D6D5D4D3D2A2
:1001E000D2D1D0CECDCCCBCAC9C7C6C5C3C2C1BF80
:1001F000BEBCBBB9B8B6B4B3B1AFAEACAAA8A7A5E4
:10020000A3A19F9E9C9A98969492908E8C8A89879F
:100210008583817F7D7B79777573716F6D6B69687D
:10022000666462605E5C5A5957555351504E4C4A51
:100230004947454342403E3D3B3A383635333230FC
:100240002F2D2C2A292826252322FFAA7F5540005E
:100250000101010101010101010202020202020287
:10026000020203030303030303030404040404045A
:100270000405050505050606060606070707070720
:1002800008080808090909090A0A0A0B0B0B0C0CD3
:100290000C0D0D0D0E0E0E0F0F0F1010111111126F
:1002A0001213131414151516161717181819191AEE
:1002B0001A1B1B1C1D1D1E1E1F2020212222232451
:1002C00024252626272829292A2B2C2D2D2E2F3090
:1002D000313232333435363738393A3B3C3D3E3FA4
:1002E000404142434445464748494A4C4D4E4F5091
:1002F000515354555658595A5B5D5E5F616264654F
:100300006668696B6C6D6F7072737577787A7B7DD8
:100310007E8082838587888A8C8E8F91939596982C
:100320009A9C9EA0A2A3A5A7A9ABADAFB1B3B5B748
:10033000BABCBEC0C2C4C6C9CBCDCFD1D4D6D8DB1F
:10034000DDDFE2E4E7E9EBEEF0F3F5F8FAFDFF0EAE
:1003500003540065006E006E006900650000000A2D
:10036000034A00730063006B0000000403090409E2
:10037000023B00020100A0FA090400000103010190
:100380000009211101000122400007058103080036
:10039000010904010001030000000921110100010D
:1003A000227B0007058203200001120100020000E9
:1003B0000008EE1E131301000102000105010902ED
:1003C000A10185020901A1000509190129081500EB
:1003D0002501950875018102050109300931158152
:1003E000257F95027508810609381581257F9501BD
:1003F00075088106050C0A38021581257F9501755F
:10040000088106C0C005010980A101850319012AE0
:10041000B700150126B700950175108100C0050CC5
:100420000901A101850419012AA002150126A002D3
:10043000950175108100C005010906A10105071984
:10044000E029E715002501950875018102950175E0
:100450000881010507190029FF150026FF009506F0
:100460007508810005081901290595057501910296
:10047000950175039101C00011241FBECFEFDAE092
:10048000DEBFCDBF11E0A0E0B1E0E4E3F3E502C0E0
:1004900005900D92AA3BB107D9F722E0AAEBB1E093
:1004A00001C01D92A338B207E1F70E94B5120C9467
:1004B00098290C94000081E0089581E008950C943F
:1004C0005D0208950C9461021F93CF93DF9300D0D7
:1004D00000D01F92CDB7DEB749835A836B8330912A
:1004E000BD0189819A81311114C0662359F02223FC
:1004F00049F00E941A09182F682F89819A810E9459
:10050000C50803C00E94EF08182F69817A81812FE6
:1005100004C00E941A0969817A810F900F900F9090
:100520000F900F90DF91CF911F910C943F10FC0121
:10053000262F408151816281738184810C946402F1
:1005400081E00895CF93DF93EC0160E00E94970271
:10055000BE01DF91CF910C9462020C9484110C9433
:10056000801108950E946F070E94B1022FEF84E36B
:100570009CE0215080409040E1F700C000000C94C6
:10058000D8210F931F93CF93DF938C0161E00E94DA
:100590009702EC01B8010E945F02882309F444C06D
:1005A000B801CE010E94F61F8823F1F1B801CE01F7
:1005B0000E94931C8823C1F1B801CE010E94521FF2
:1005C000882391F1B801CE010E949A1B882361F122
:1005D000F8018281882309F1CB358DE5D807C1F078
:1005E00050F4C115FCE5DF0781F0CF3DDC45A9F4EF
:1005F0000E94510E19C0CC35EDE5DE0761F0CD3516
:10060000DD4559F40E94940D08C00E94B2020CC04E
:100610000E949D0D02C00E94A00DC801DF91CF91E4
:100620001F910F910C945B0280E0DF91CF911F919D
:100630000F9108950E940D210C9433030E943603FC
:100640000C94132108950C94220381E008950C94D6
:1006500025030895CF93C82F0E9423038C2F0E9457
:100660002703CF91089580E00C942A030E94522022
:100670000C942A030E9452209091BC01891721F00A
:100680008093BC010C942A030895CF93DF93CDB7D8
:10069000DEB72B970FB6F894DEBF0FBECDBF4F83EA
:1006A000588769877A878B8761110E94E00C9E01C9
:1006B0002F5F3F4F86E0F90111928A95E9F785E0B7
:1006C000FE013796D90101900D928A95E1F7898153
:1006D0009A814C815D81452B31F09F3F31F491E04F
:1006E0008F3F19F403C091E001C090E090FF09C072
:1006F00049815A816B817C818D819E810E94010C90
:1007000005C0C9010E94A0028111F2CF2B960FB63D
:10071000F894DEBF0FBECDBFDF91CF910895FC01ED
:10072000808191810E945C090895CF93882309F408
:10073000A9C0C82F8238C1F40E94522081FDA2C0F6
:1007400069E380910201909103010E94E5200E94DB
:10075000020D2FEF81EE94E0215080409040E1F7B0
:1007600000C0000069E319C0833801F50E945220DF
:1007700080FD88C063E580910201909103010E9491
:10078000E5200E94020D2FEF81EE94E02150804081
:100790009040E1F700C0000063E580910201909174
:1007A00003010E94E720CF910C94020D8438C1F41C
:1007B0000E94522082FD66C067E480910201909100
:1007C00003010E94E5200E94020D2FEF81EE94E0CC
:1007D000215080409040E1F700C0000067E4DDCF89
:1007E0008CEF8C0F813AF8F48C2F0E94091F811135
:1007F00049C06C2F80910201909103010E94AF20AB
:10080000882349F06C2F80910201909103010E948E
:10081000E7200E94020D6C2F80910201909103014C
:100820000E94E520C0CF80E28C0F883048F4C7706A
:1008300081E001C0880FCA95EAF70E94C30CB3CFCC
:10084000EBE5EC0FE33040F4F0E0E65AFE4F808138
:1008500090E0CF910C947720E8E5EC0FE73150F46D
:10086000F0E0EE0FFF1FE45DFE4F80819181CF919C
:100870000C948D20CD3E30F08C2F0E943A13CF91F6
:100880000C940C14CF910895882309F464C0823825
:1008900079F40E94522081FF5EC069E380910201D9
:1008A000909103010E94E5200E94020D69E310C0AF
:1008B0008338B1F40E94522080FF4DC063E58091DF
:1008C0000201909103010E94E5200E94020D63E560
:1008D00080910201909103010E94E7200C94020D87
:1008E000843879F40E94522082FF35C067E48091F9
:1008F0000201909103010E94E5200E94020D67E42D
:10090000E7CF9CEF980F913A10F4682FE1CF90E277
:10091000980F983050F4877091E001C0990F8A9534
:10092000EAF7892F0E94C90CD9CF9BE5980F933025
:1009300020F480E090E00C94772098E5980F9731B0
:1009400020F480E090E00C948D208D3E20F00E94F9
:1009500095130C940C1408951F93CF93DF93182FC5
:10096000EB010E949503209741F08FE99FE00197EA
:10097000F1F700C000002197F6CF812FDF91CF91D2
:100980001F910C944404893319F060E070E002C0B8
:1009900060E570E00C94AC04882321F00E94C30C45
:1009A0000C94020D0895882321F00E94C90C0C9428
:1009B000020D0895CF92DF92EF92FF920F931F9353
:1009C000CF93DF937C01D62FC72FFC0112810581C5
:1009D00002950F700E94B90C8823B9F01123A9F079
:1009E0008C2F807F803421F080E28D0F883068F07A
:1009F0008091620282FD09C082E00E94620D0E9425
:100A0000B90C91E0D82ED92601C0D12CCC2EC2949D
:100A10008FE0C8228C2D90E08C30910508F0CFC17A
:100A2000FC01EA5AFF4F0C94FF288C2F807FCF7077
:100A3000882311F0C295C07F112399F0CC2309F4CB
:100A4000AAC180E28D0F883010F0D11104C08C2F24
:100A50000E94C30C03C08C2F0E94D30C0E94020D75
:100A60009AC18D2F0E944404CC2309F4A8C180E2CE
:100A70008D0F883038F1DD2329F18C2F0E94D90C9D
:100A800024C08C2F807FCF70803211F0C295C07F40
:100A9000DD2319F0D130A1F13DC08091620282FFC7
:100AA00017C0112349F0CC2329F08C2F0E94C30CCE
:100AB0000E94020D80E070C180E00E944404CC23BB
:100AC00009F47DC18C2F0E94C90C0E94020D77C1D0
:100AD000112371F0002341F0013031F40E94E30C46
:100AE0008C2B0E94EB0C6BC10E94E30C8C2B1DC065
:100AF000002319F0013009F462C10E94F80C25C0EE
:100B0000112321F0033008F05AC10EC0023008F062
:100B100056C11BC0112361F0002331F0F70185811C
:100B200080FF39C18F7085838C2F0E94CC0447C110
:100B3000002359F0D93309F03FC1FFEF07EE13E06E
:100B4000F15000401040E1F735C18C2F0E94D304D2
:100B500036C18C2F86958695837019F0813061F0AF
:100B60002EC1112321F08D2F9C2F937002C080E0A5
:100B700090E00E9477202BC1112321F08D2F9C2F14
:100B8000937002C080E090E00E948D2020C18D2FE4
:100B9000112319F00E943A1302C00E9495130E947B
:100BA0000C1415C18C2F837009F047C011110BC1B3
:100BB0002D2F229526952770220F220F6D2F6F70F3
:100BC000862F90E0A0E0B0E0022E04C0880F991FAD
:100BD000AA1FBB1F0A94D2F7D4FF10C04FE050E009
:100BE00060E070E004C0440F551F661F771F2A9510
:100BF000D2F7409550956095709503C040E050E065
:100C0000BA01C695C695C3708A019B01082B192BA2
:100C10002A2B3B2BC901B801C23049F058F4C1302E
:100C200019F00E94DB07CFC00E94C907CCC00E9408
:100C3000ED07C9C00E94C707C6C0112319F08C2F49
:100C4000817001C08695882309F4BDC02D2F22959F
:100C500026952770220F220F6D2F6F70862F90E040
:100C6000A0E0B0E0022E04C0880F991FAA1FBB1F8E
:100C70000A94D2F7D4FF10C04FE050E060E070E07B
:100C800004C0440F551F661F771F2A95D2F7409561
:100C900050956095709503C040E050E0BA01C6954C
:100CA000C695C3708A019B01082B192B2A2B3B2B5D
:100CB000C901B801C23049F058F4C13019F00E949E
:100CC000A00881C00E948E087EC00E94B2087BC02E
:100CD0000E94010878C0CF70112339F08C2F0E9438
:100CE00027088D2F0E94CC046EC08D2F0E94D30444
:100CF0008C2F0E94480867C0D23F21F128F4D03FD2
:100D000041F0D13FC1F043C0D33F19F1D43F79F056
:100D10003EC0112341F0023008F051C08C2F8F717A
:100D20000E946D084CC0033008F049C0F7CF809195
:100D3000620282FF18C0112339F08C2F8F710E943C
:100D400027083DC01123C9F38C2F8F710E944808DA
:100D500036C0112329F08C2F8F710E9412082FC0EA
:100D60000E940D082CC0112349F0CF718C2F0E94D6
:100D7000270863E08C2F0E94470D21C081E00E946C
:100D8000620D0230E0F082E00E94620D18C0112373
:100D900031F0002391F28D2F0E94950310C00023A3
:100DA00099F2D93349F41FEF27EE33E01150204078
:100DB0003040E1F700C000008D2F0E94440488EF0E
:100DC0008C0D843020F40E9452200E942A03DD20E2
:100DD000C9F00E94B50C80FD15C0F70112820E9477
:100DE000AF0C0E942708C7010E9423070E94AF0C86
:100DF000DF91CF911F910F91FF90EF90DF90CF90F7
:100E00000C944808DF91CF911F910F91FF90EF90C4
:100E1000DF90CF9008950F931F93CF93DF93EC0152
:100E2000688179818A810E9467098C010E94C408C7
:100E30000E94B507B801CE010E94DA04DF91CF917C
:100E40001F910F910895CF93DF93EC0198818981D1
:100E50002B813C81232B31F08F3F31F481E09F3F88
:100E600019F403C081E001C080E080FD1DC0CE0107
:100E70000E94C102811110C00E94B90C8823A1F008
:100E80008A81882389F08091620282FD0DC082E010
:100E9000DF91CF910C94620DCE010E940B07CE0121
:100EA000DF91CF910C94A202DF91CF91089580E061
:100EB00090E00E94772080E090E00E948D200E94C8
:100EC000E00C0E94020D0E943D150C940C148091C0
:100ED0000201909103010E94E9200C9457070E949F
:100EE000D00C0C94670792959F70963079F010F4AF
:100EF000925001C09A50923068F4803F69F018F423
:100F0000883E40F409C0843F29F406C0883E20F0A2
:100F1000813F11F080E0089581E00895FC01808117
:100F200091810E945C090E9473070895CF93DF931B
:100F300000D000D01F92CDB7DEB70F900F900F906A
:100F40000F900F90DF91CF910895CF93DF9300D052
:100F500000D000D0CDB7DEB726960FB6F894DEBF2E
:100F60000FBECDBFDF91CF910895089508950C94E1
:100F7000B6070C94B7070E94B9076093CC01709331
:100F8000CD018093CE019093CF010C9457070C9420
:100F9000BB070F931F930091CC011091CD012091BD
:100FA000CE013091CF01602B712B822B932B1F919F
:100FB0000F910C94BB070F931F930091CC011091DC
:100FC000CD012091CE013091CF0160237123822386
:100FD00093231F910F910C94BB070F931F930091C4
:100FE000CC011091CD012091CE013091CF0160272D
:100FF0007127822793271F910F910C94BB070C94A4
:10100000B6070E94FF076093C8017093C9018093DF
:10101000CA019093CB010C94570760E070E0CB01BC
:101020000C9401080F931F9341E050E060E070E0E2
:101030008A019B0104C0000F111F221F331F8A95D4
:10104000D2F7C901B8011F910F910C9401080F93B9
:101050001F9341E050E060E070E004C0440F551F72
:10106000661F771F8A95D2F78091C8019091C901B8
:10107000A091CA01B091CB018A019B01082B192BC9
:101080002A2B3B2BC901B8011F910F910C94010829
:101090000F931F9341E050E060E070E004C0440F04
:1010A000551F661F771F8A95D2F74095509560951A
:1010B00070958091C8019091C901A091CA01B09129
:1010C000CB018A019B01082319232A233B23C90151
:1010D000B8011F910F910C9401080F931F9341E0E9
:1010E00050E060E070E004C0440F551F661F771F9A
:1010F0008A95D2F78091C8019091C901A091CA0147
:10110000B091CB018A019B01082719272A273B2789
:10111000C901B8011F910F910C9401080F931F93FF
:101120000091C8011091C9012091CA013091CB01F1
:10113000602B712B822B932B1F910F910C94010824
:101140000F931F930091C8011091C9012091CA010A
:101150003091CB0160237123822393231F910F9140
:101160000C9401080F931F930091C8011091C901BD
:101170002091CA013091CB016027712782279327E4
:101180001F910F910C9401080895990F990F890FE1
:10119000E82FE695E695E695877051E001C0550F7A
:1011A0008A95EAF785E0E89FF0011124E254FE4FAA
:1011B00020E030E070E04081CB01022E02C0969525
:1011C00087950A94E2F78170819584278523842787
:1011D00081932F5F3F4F2530310569F70895990FAF
:1011E000990F890F682F669566956695982F977069
:1011F00085E0689FB001112440E050E080E0FB01F1
:10120000E40FF51FE254FE4F208130E0092E02C0AA
:10121000369527950A94E2F721703327042E01C0F2
:10122000220F0A94EAF7822B4F5F5F4F453051053A
:1012300031F70895BF92CF92DF92EF92FF920F9312
:101240001F93CF93DF938C01C090C801D090C90148
:10125000E090CA01F090CB018091CC019091CD013A
:10126000A091CE01B091CF01C82AD92AEA2AFB2A3F
:10127000CFE1D0E0D701C6010C2E04C0B695A795EA
:10128000979587950A94D2F780FD04C0219790F72F
:10129000B12C07C0BC2EB8018C2F0E9454100197AE
:1012A000A9F38B2DDF91CF911F910F91FF90EF90BC
:1012B000DF90CF90BF900895CF93DF93EC010E9411
:1012C0001A09BE010E945410DF91CF9108951F9317
:1012D000CF93DF93EB019091BD01992321F0CB01D6
:1012E0000E945C0913C0882349F0CB010E941A09AF
:1012F000182F682FCE010E94C50804C0CB010E94A0
:10130000EF08182FBE01812F0E945410DF91CF915A
:101310001F9108951F93CF93DF93C091D00116E0E2
:101320008091D101C81799F0D0E01C9FF0011D9F5A
:10133000F00D1124EE52FE4F408151816281738184
:10134000848195810E94A5072196C770E9CFDF911E
:10135000CF911F9108954091020250910302609134
:1013600004027091050280910602909107020C948C
:10137000A507EF92FF920F931F93CF93DF93809176
:10138000070282958F7009F065C08091040288235E
:1013900009F460C08091D001F090D1011091020257
:1013A00000910302609105027091060291E01F3FD7
:1013B00009F090E0C0910001D0910101292F96E041
:1013C000E92E8F1509F446C06115710521F00F3F14
:1013D00021F030E003C031E001C0322F90E030FD59
:1013E00036C0E89EF001E99EF00D1124DF01AE52F7
:1013F000BE4F11963C911197301329C03C91311387
:1014000026C012963C911297311121C013964D912E
:101410005C911497461B570B4C175D07C0F48091E5
:1014200007028F70806180930702E952FE4F80812E
:101430008F708061808382E092E00E942307DF91B9
:10144000CF911F910F91FF90EF900C948A09019614
:101450008770B7CFDF91CF911F910F91FF90EF90E1
:1014600008959F92AF92BF92CF92DF92EF92FF9238
:101470000F931F93CF93DF93CDB7DEB761970FB66E
:10148000F894DEBF0FBECDBF8C0185E0F801DE0110
:101490001D9601900D928A95E1F7D8011296EC9075
:1014A00090910202E0910302209105023091060220
:1014B0002115310531F0EF3F31F481E09F3F19F400
:1014C00003C081E001C080E0B82FB1709B2E80FD89
:1014D00047C1D8014C9111965C9111971396AD902C
:1014E000BC90149782E0C82E82E0D82EF0900402BF
:1014F000B501621B730B2091000130910101FF20A7
:1015000009F4D9C0809107026217730708F095C0EB
:10151000282F207F09F052C05E1313C0491311C059
:10152000FE2CE1100EC08F708061809307020E9434
:10153000AB09C6010E94230780910702F801858349
:101540004DC1AB2831F05F3F31F481E04F3F19F4DA
:1015500003C081E001C080E080FD03C081E08E25F2
:1015600002C080E090E0F82FF170FF2E80FF1CC0D9
:101570008091D0012091D10136E0821709F40BC18E
:1015800090E0389FF001399FF00D1124EE52FE4F8C
:101590006181561306C06081461303C06281E61262
:1015A00003C001968770E9CFFE2CEE2009F416C126
:1015B0008091070281608093070254C05E1306C0C9
:1015C000491304C0E11002C0F80199C0C8010E948B
:1015D0008E07882361F1EE2051F120910702822FBE
:1015E00082958F7090E0029774F080910202909142
:1015F000030298878F831986BB86AA862C87CE0123
:1016000007960E94230786E0F801A2E0B2E001906D
:101610000D928A95E1F70E94B9090E94AB090AC0B0
:101620005E1711F1C8010E948E0781112CC0C801FC
:101630000E942307FF24F394D1C0282F207F81F735
:101640007A2DB98AA88A6E2D89890E94960782E030
:1016500092E00E94230786E0D6011D928A95E9F761
:101660000E94AB09F12CBAC04913DCCFE110DACFEC
:10167000F8018583C8010E94230786E0D6011D92E8
:101680008A95E9F7ABC0EE2091F220910702822FF4
:1016900082958F7090E002970CF4B5CF8091020292
:1016A000909103029A8389831B82BD82AC822E8330
:1016B000CE010196A6CF6217730708F044C0FE2C36
:1016C000EE2009F4B4CF5E1330C049132EC0209130
:1016D000070220FD21C0822F82958F70482F50E095
:1016E00041155105C9F0F80125834F30510541F0EE
:1016F0008F5F982F9295907F822F8F70892B858393
:10170000C8010E94230786E0F801A2E0B2E0019040
:101710000D928A95E1F73CC086E0F801A2E0B2E0C4
:1017200001900D928A95E1F759C0C8010E948E0779
:10173000811169CF80910702816080930702C801FF
:101740000E9423074BC07A2DB98AA88A6E2D8989F9
:101750000E94960786E0D6011D928A95E9F718C087
:10176000EE2009F464CFC8010E948E07F82E88236A
:1017700009F45DCF86E0F801A2E0B2E001900D929D
:101780008A95E1F782E092E00E948F030E94B909F6
:101790000E94AB0923C04D875E878D859E850E9480
:1017A0005C09292F22952F70223028F49F7039F080
:1017B000811105C00BC0243028F49F7049F4805E6D
:1017C000883020F0C8010E9423079F2CF92C06C006
:1017D000D80115969C91907F91F7F8CF8F2D619647
:1017E0000FB6F894DEBF0FBECDBFDF91CF911F9132
:1017F0000F91FF90EF90DF90CF90BF90AF909F90B0
:1018000008951F93CF93DF93CDB7DEB72C970FB614
:10181000F894DEBF0FBECDBF4F83588769877A87A4
:101820008B879C87CE0107960E94310A8823D1F0CE
:101830009F8188852A853B85232B31F08F3F31F4AA
:1018400081E09F3F19F403C081E001C080E080FD8A
:1018500047C04F81588569857A858B859C850E9414
:10186000A5073EC086E0FE013796DE011196019085
:101870000D928A95E1F7FF81E8856A857B85611580
:10188000710531F0EF3F31F481E0FF3F19F403C0FF
:1018900081E001C080E080FD23C02091D10130E0D3
:1018A000C9010196877099274091D00150E08417B3
:1018B0009507F1F1F983EA837D836C8396E0929F2B
:1018C000D001939FB00D1124AE52BE4FFE01319650
:1018D00001900D929A95E1F78093D1010E948A09B7
:1018E00016E08091D0019091D101891771F1189F74
:1018F000C00111248E529E4F0E94310A882329F183
:10190000E091D0011E9FF0011124EE52FE4F408164
:10191000518162817381848195810E94A5078091A4
:10192000D00190E00196877099278093D001D9CF9C
:101930000E946F071092D1011092D001E2E0F2E014
:1019400086E0DF011D928A95E9F72C960FB6F89490
:10195000DEBF0FBECDBFDF91CF911F910895809163
:101960001002859585958595089580911002877060
:10197000089590911002977081E009F480E0089535
:1019800080911B02089590911B02892B80931B026A
:101990000895809590911B02892380931B020895DE
:1019A00010921B02089590911A02892B80931A02BB
:1019B0000895809590911A02892380931A020895C0
:1019C00010921A02089580911102089508950C94BE
:1019D000E60C0C94E70C9091620292FD08C0909185
:1019E0001102981721F0809311020C94E90C0895CC
:1019F00080911102882329F01092110280E00C944A
:101A0000E90C0895CF93DF93E0910201F091030177
:101A100080911B028083E0910201F091030190818B
:101A200080911A02892B808380911102882381F092
:101A3000E0910201F09103019081892B80838091D4
:101A40000201909103010E94A32081110E94F80CD1
:101A5000C0910201D091030148E050E068E072E0DB
:101A6000CE010E944329892B69F088E0FE01A8E09D
:101A7000B2E001900D928A95E1F7CE01DF91CF910E
:101A80000C945E20DF91CF9108950C94E60C909118
:101A9000620292FD10C098E0899F90011124262BCC
:101AA000209310020E942708809110028595859549
:101AB00085950C94450D0C9427081092100280E037
:101AC0000C94450D20911002809582238093100282
:101AD000982F977099F430E0482F082E000C550B82
:101AE0002417350759F09091620292FD07C0859541
:101AF000859585950E9448080C945D0D08959091F8
:101B0000620292FB222720F9281769F080FB92F9E4
:101B10009093620280916102909162020E94CD0DC9
:101B200082E00C94620D08958091620282FB882706
:101B300080F991E089270C947F0D81E00C947F0D52
:101B400080E00C947F0D6FEF7FEF80E090E00C94CD
:101B5000822980E090E00E945E2921E0893E9E4F2C
:101B600009F020E0822F089582E090E00C94502943
:101B700083E090E00C945029CF9384E090E00E94A1
:101B80005029C82F82E290E00E9450292C2F30E08B
:101B9000A901582BCA01CF910895CF93C92F682F5F
:101BA00084E090E00E9464296C2F82E290E0CF9163
:101BB0000C946429AB01BC018FE090E00C94762971
:101BC000AB01BC0183E190E00C94762960E070E009
:101BD000CB010C94E00D60E070E0CB010E94DA0DC7
:101BE0000C94E60D69EE7EEF80E090E00E94822981
:101BF00060E082E090E00E94642960E083E090E091
:101C00000E9464291092CC011092CD011092CE0155
:101C10001092CF0160E084E090E00E94642960E0CF
:101C200082E290E00E94642960E085E090E00E94FA
:101C3000642960E086E090E00E9464296FEF87E00D
:101C400090E00E94642940E050E0BA0188E090E012
:101C50000E94762960E08DE090E00E94642940E0D7
:101C600050E0BA0188E190E00E94762960E087E1C7
:101C700090E00E94642940E050E0BA018CE190E0DD
:101C80000E94762960E070E080E290E00E94822964
:101C900040E050E0BA0188E190E00E9476290C947F
:101CA000EB0D0C94F20D682F8EE090E00C946429FB
:101CB0000E9497216093230270932402809325024F
:101CC0009093260260931F0270932002809321025A
:101CD00090932202089585B7806885BF85B7806894
:101CE00085BF089581E008950C94720E08950C94B8
:101CF000760E0C94760E0C94790E0C94760E0C9451
:101D00007D0E0C94760E0E946B0E80E391E10E9492
:101D100048200E94810E0C947F0E0E94770E0C9436
:101D2000760E0E944A110C9429030E9482210E947F
:101D30001A120E94910E0E94B91A0C947B0E8F9277
:101D40009F92AF92BF92CF92DF92EF92FF920F934A
:101D50001F93CF93DF93CDB7DEB72A970FB6F894D2
:101D6000DEBF0FBECDBF0E942F12982E81110E94A0
:101D7000580E8CE1A82E82E0B82E00E010E0802EF4
:101D8000802F0E946E11D82EF501C1905F01C826E8
:101D9000B1F40F5F1F4F0330110589F78FEF89836F
:101DA0008A831B820E948B218160782F9D838C8384
:101DB00049815A816B818D810E9445032FC080919A
:101DC000270281FD0E947411E12CFF24F3948C2DD5
:101DD0008F21F1F00E94740E882399F0EE828F8299
:101DE000DF2081E009F480E088870E948B218160F8
:101DF000782F9A8789874E815F8168858A850E94BE
:101E00004503F801E45EFD4F8081F826F08206C0AC
:101E1000E394FF0CF4E0EF12DACFBBCF81E0911036
:101E200001C080E02A960FB6F894DEBF0FBECDBF8A
:101E3000DF91CF911F910F91FF90EF90DF90CF90A6
:101E4000BF90AF909F908F9008950E949F0E0E9428
:101E5000EC1A0E942A140C943A03CF93DF930E9449
:101E60005910EC01811521E5920708F045C0811554
:101E700030E5930708F094C0883E910528F5803E30
:101E8000910508F0F8C0883A910570F4853A9105FB
:101E900008F07CC08130910509F475C008F4E8C0F1
:101EA000049708F0E8C0E4C08F3B910508F0E0C05B
:101EB000C85AD0E0CC0FDD1FC35ADE4F0990D8813D
:101EC000C02DCE019464D8C0811540E2940758F427
:101ED000811551E0950708F0CEC08D3E910508F4BC
:101EE000C7C09065C9C0C11580E4D80708F4C0C058
:101EF000DF70CE01906AC0C0811525E59207A8F475
:101F0000811534E5930708F095C0811543E59407E2
:101F100008F07BC0811552E5950708F061C0D82F05
:101F2000CC27CE01816F906AA7C0C11589E5D8077B
:101F3000A0F4C11528E5D20708F082C0C11536E526
:101F4000D30708F095C08C2F0E94ED108F7190E0A0
:101F5000D82FCC27CE0190628FC0C1154AE5D40797
:101F600008F474C0CE0190568115904208F080C0EC
:101F70008D2F8F710E94ED10DD27D0628F71AE0121
:101F8000582BCA0179C081E090E076C0C55AD0E0F4
:101F9000C557DE4F8881C82FD0E0CE0190646CC059
:101FA00074E0969587957A95E1F7282F23703C2F5A
:101FB000337081E090E002C0880F991F3A95E2F7F4
:101FC0009C68AC01522B9A019C2F9F709695969518
:101FD00050E2959FE0011124C9018C2B9D2B4CC030
:101FE0008370992721E030E002C0220F331F8A95C9
:101FF000E2F79C2F9695969580E2989FE001112438
:10200000C22BD32BCE019C6837C08370992721E067
:1020100030E002C0220F331F8A95E2F79C2F96957D
:10202000969540E2949FE0011124C22BD32BCE0160
:102030009A6822C0D82FCC27CE01846F906A1CC02A
:10204000DC2FCC27CE01806F906A16C08C2F8F704A
:102050000E94ED1094E0D695C7959A95E1F7CF7060
:10206000D0E0DC2FCC27D0699E01282BC90104C009
:1020700080E090E001C0CE01DF91CF91089590E023
:10208000FC01EE0FFF1FE80FF91FE70FF11DEE0F28
:10209000FF1FEE0FFF1FE60FF11DEE0FFF1FE852AF
:1020A000FF4F8591949108950E943F100E942D0F3B
:1020B00008958238910569F1B0F48133910509F4EE
:1020C0006DC048F48932910509F463C08A329105E4
:1020D00009F469C008958533910509F455C0893321
:1020E0009105B9F00895833E910569F138F4803E79
:1020F0009105B1F0823E910509F10895863E910562
:10210000A9F1873E9105B9F1843E910509F064C0BB
:1021100023C02091610220FD4FC021FD4DC00895D4
:102120008091610280FD44C08091620280FF44C0C2
:102130008091610284FD42C083EE4DC080916102B6
:1021400082FF38C0F5CF8091610282FD33C080915B
:10215000620280FD31C0ECCF8091620281FF32C00B
:102160008091610284FD2AC087EE35C080916102B2
:1021700083FF26C0F5CF8091610283FD21C080914D
:10218000620281FD1FC0ECCF8091610285FD1CC001
:102190001DC08091610285FD19C016C08091610249
:1021A00086FD16C017C08091610286FD13C010C065
:1021B00089E311C082EE0FC080EE0DC080E00BC03D
:1021C00086EE09C084EE07C089E205C085E303C03E
:1021D0008AE201C081E390E008959091610292FF4C
:1021E0000DC0282F2871283019F4877F846006C01D
:1021F000282F2471243011F48B7F886093FF0DC049
:10220000282F2871283119F4877E846106C0282F71
:102210002471243111F48B7E88612091620220FFA9
:102220000DC0382F3871383019F4877F816006C0AF
:10223000382F3171313011F48E7F886021FF0DC04D
:10224000282F2871283119F4877E816106C0282F34
:102250002171213111F48E7E886194FD877E08956D
:1022600080E008950C94A30D0E942F128FE39CE947
:102270000197F1F700C000000E942F1280E00E9439
:102280006E1180FF04C00E9432110C94D821089571
:102290000C9434110E94A90D811102C00E94510EAC
:1022A0000E94B40D809327020E94BC0D909362029D
:1022B000809361020E9448110E94B80D682F70E05F
:1022C00080E090E00E94C7076091C8017091C90149
:1022D0008091CA019091CB010C94FF07E82FF0E0A8
:1022E000EA59FD4F80810895089580EA8A95F1F7B3
:1022F000089500C008950C94751108950C947D11F3
:102300000C947E110C947D110C948211F894E82F9A
:10231000E295EF70F0E031A1282F2F7081E090E07E
:1023200001C0880F2A95EAF7982F9095932391A3DF
:1023300092A1892B82A378940895CF93DF9386E6A8
:102340000E94861184E90E94861180E90E9486110C
:10235000CEE8D1E089918F3F11F00E94861181E093
:10236000C239D807B9F7DF91CF910895CF92DF92A4
:10237000EF92FF920F931F93CF93DF938C01C62FA1
:10238000D0E0CE018E569E4F7C01FC0190819F3F94
:1023900009F447C0D62EF894E92FE295EF70F0E0EB
:1023A00081A19F7021E030E001C0220F9A95EAF7E9
:1023B000822B81A382A12095282322A378940E94B6
:1023C0007911EEE8F1E042E951E031E0C12C2191D0
:1023D0002F3F89F0A22FA295AF70B0E090968C911C
:1023E00090E02F7002C0959587952A95E2F780FDC1
:1023F00002C0832F01C080E0C82A330F4E175F0749
:1024000031F7F70180818F3F11F00E94861161E062
:10241000C11001C060E08D2D0E947B11C00FD11F43
:10242000C882DF91CF911F910F91FF90EF90DF90C5
:10243000CF9008950E949D1183E0E6E6F2E0DF016F
:10244000982F1D929A95E9F7E3E6F2E0DF011D92DD
:102450008A95E9F783E00E9472120C94AD021F93F3
:10246000CF93DF9300D01F92CDB7DEB719821A82C7
:102470001B8260E0CE0101960E94B61161E0CE01A0
:1024800001960E94B61162E0CE0101960E94B6113B
:1024900043E050E0BE016F5F7F4F83E692E00E9411
:1024A000432911E0009709F410E0892B49F0898154
:1024B0009A81AB818093630290936402A09365023A
:1024C000212F43E066E672E083E692E00E947312F9
:1024D0000E94AF02812F0F900F900F90DF91CF914C
:1024E0001F9108950895FF920F931F93CF93DF9349
:1024F0008C01F62ED72FC42F222349F081E0809340
:102500002A020E948B2190932902809328028091B5
:102510002A028823C1F080912802909129020E940A
:10252000A321059780F0EF2DFD2FD8014C2F50E00F
:10253000CD01801B910B841795071CF48D9181931D
:10254000F7CF10922A02DF91CF911F910F91FF9048
:1025500008950E947B230E94950E0C9487230E946D
:102560008B230E94250F0C94A5230E9429210E94F1
:1025700062230E94830E0E94A9120E94AF120E9441
:102580008D0EFBCF8091310280FF06C06091090162
:1025900070E0660F771F26C081FF04C060910901BB
:1025A00084E005C082FF07C06091090188E0689F50
:1025B000B001112417C0909130029923D1F060919D
:1025C0000801961788F72091090188E0289F90015B
:1025D0001124929FA001939F500D112470E0CA0115
:1025E0000E94C9286038710540F46115710519F41D
:1025F00006C068E070E0862F08958FE7089581E0B7
:1026000008958091310280FF08C06091050170E05B
:10261000759567957595679521C081FF06C0609196
:10262000050170E07595679519C082FF04C060913F
:10263000050170E010C090912F02992399F06091EC
:1026400004019617A0F780910501899FC00111240C
:1026500070E00E94C9286038710540F46115710569
:1026600019F406C061E070E0862F08958FE70895A1
:1026700081E008958D3E21F40E94C212819504C02C
:102680008E3E29F40E94C2128093350208958F3E37
:1026900021F40E94C212819504C0803F29F40E9457
:1026A000C212809334020895893F19F40E940113E5
:1026B00005C08A3F31F40E94011381958093360250
:1026C00008958B3F21F40E940113819504C08C3F33
:1026D00029F40E9401138093370208959FE0980F18
:1026E000983078F421E030E0A90102C0440F551F72
:1026F0009A95E2F7CA0190913302892B80933302B5
:1027000008958D3F21F48091310281600BC08E3F8E
:1027100021F480913102826005C08F3F29F48091BD
:10272000310284608093310208958D3E39F4909196
:10273000350297FF35C01092350259C08E3E29F4FC
:10274000909135021916BCF32BC0909134028F3E44
:1027500029F497FF25C01092340249C0803F19F434
:102760001916CCF31DC090913602893F29F4191631
:10277000BCF4109236023BC08A3F19F497FF10C098
:10278000F8CF8B3F39F49091370297FF09C0109230
:1027900037022DC08C3F21F4909137021916BCF3FB
:1027A0009FE0980F983080F421E030E0A90102C04A
:1027B000440F551F9A95E2F7CA0180959091330214
:1027C00089238093330213C08D3F21F4809131021D
:1027D0008E7F0BC08E3F21F4809131028D7F05C02A
:1027E0008F3F29F4809131028B7F80933102809159
:1027F0003402811106C080913502811102C010920D
:10280000300280913602811106C080913702811119
:1028100002C010922F0208950E948B212091340251
:10282000211104C020913502222321F090932E0221
:1028300080932D0220913602211104C0209137028D
:10284000222321F090932C0280932B0282E392E0CA
:102850000C946920EF92FF920F931F93CF93DF9315
:1028600000D000D000D0CDB7DEB786E0E2E3F2E0E2
:10287000DE01119601900D928A95E1F7E090340205
:10288000F090350200913602109137021092340216
:10289000109235021092360210923702E11003C0F6
:1028A000FF2009F45DC080912D0290912E020E94BC
:1028B000A321AC0190913002992339F020910A01B3
:1028C00030E02417350758F04BC020910B018AE007
:1028D000289F900111242417350718F041C09F3F0D
:1028E00019F09F5F90933002EE2061F00E94C212B7
:1028F0001E1414F09FEF01C091E0989F902D1124B9
:1029000090933402FF2061F00E94C2121F1414F051
:102910009FEF01C091E0989F902D11249093350274
:10292000309134023323E1F0209135022223C1F0AB
:1029300045EB3403C0011124992319F0909334021C
:1029400003C081E08093340235EB2303C0011124DE
:10295000992319F09093350203C081E080933502EA
:10296000011103C0112309F45DC080912B029091E5
:102970002C020E94A321AC0190912F02992339F0DF
:102980002091060130E02417350758F04BC0209104
:1029900007018AE0289F900111242417350718F0B9
:1029A00041C09F3F19F09F5F90932F02002361F079
:1029B0000E940113101614F09FEF01C091E0989F40
:1029C000902D112490933602112361F00E9401137F
:1029D000111614F09FEF01C091E0989F902D1124E3
:1029E00090933702309136023323E1F02091370281
:1029F0002223C1F045EB3403C0011124992319F0BF
:102A00009093360203C081E08093360235EB2303B6
:102A1000C0011124992319F09093370203C081E07B
:102A2000809337028091340281110BC0809135026E
:102A3000811107C080913602811103C08091370255
:102A400081110E940C14EB82FC820D831E8386E0B0
:102A5000FE013196A2E3B2E001900D928A95E1F772
:102A600026960FB6F894DEBF0FBECDBFDF91CF9193
:102A70001F910F91FF90EF900895E2E3F2E086E05E
:102A8000DF011D928A95E9F71092300210922F0211
:102A9000109231020895EF92FF920F931F93CF93FC
:102AA000DF938B01682F11110AC0442329F0E82F0E
:102AB000F0E0E15BFD4F6491762F862F75C0212FEA
:102AC00030E0E82FF0E0442321F0E15BFD4FE4919A
:102AD000F0E046E0049FC0011124CFEFD0E0BE013A
:102AE0000E94B5284BEA4603C001479F900D112470
:102AF000800F911D800F911D982F990F890FAE01A6
:102B0000421B530B4E9FD0014F9FB00D5E9FB00DE7
:102B100011249B2F189FA0011124452F55278E01AA
:102B2000041B150B0E9FA0010F9F500D1E9F500DF3
:102B300011247E01E81AF108E29E8001E39E100D47
:102B4000F29E100D1124212F3327C21BD30BCE9FD1
:102B50009001CF9F300DDE9F300D11246230710542
:102B6000A9F048F46115710569F061307105C9F487
:102B70008B2F752F0DC06430710581F058F06630D1
:102B8000710579F47E2F8B2F932F0DC0832F7B2F10
:102B90009E2F09C08E2F7B2F952F05C08E2F732F50
:102BA00002C07E2F852F692FDF91CF911F910F914A
:102BB000FF90EF90089541E00E944B150895FC01AD
:102BC000828120813181982F281708F4922F39179C
:102BD00008F4932F9383391B3183291B2083891B8E
:102BE0008283089508950E94DB150895CF93DF93A3
:102BF000762FE901682F842F0E94F315798368836B
:102C00008A831B82DF91CF91089580916902282FDA
:102C1000269530E02115310519F48170826005C0D8
:102C20002532310524F0817088648093690208950B
:102C300088E090E00C945829CF92DF92EF92FF92B7
:102C40006B017C010E940516B701A60188E090E0A7
:102C5000FF90EF90DF90CF900C947629E9E6F2E0B8
:102C600083E0808311828FEF82838383148260816B
:102C70007181828193810C941C168091690280FF7E
:102C800002C08695089580E0089590916D0293307A
:102C900018F49F5F90936D02882351F06091690250
:102CA00070916A0280916B0290916C020C941C16D8
:102CB000089581E00C94451690916D02992319F0C6
:102CC000915090936D02882351F060916902709148
:102CD0006A0280916B0290916C020C941C1608950C
:102CE00081E00C945C1670E00C94691CEF92FF92EA
:102CF0000F931F93CF93DF9300911001809169028E
:102D000080FF0BC0C0910F0124E0C29FE00111249D
:102D1000C259DD4F7E0110E012C0809111019091E7
:102D20001201891778F724E0829FF0011124E259FB
:102D3000FD4F11821082128213828F5FF2CF101723
:102D400041F0C7010E94DF151F5F84E0E80EF11C0F
:102D5000F6CF612FCE01DF91CF911F910F91FF90A0
:102D6000EF900C9473169091690290FF14C09091AB
:102D7000110120911201921760F434E0939FF00149
:102D80001124E259FD4F81836083428313829F5F48
:102D9000F2CF0C9476160895CF93DF9300D000D035
:102DA000CDB7DEB79091690290FF0AC09E012F5FF8
:102DB0003F4F0E94F6154B8169818A810E94B316AC
:102DC0000F900F900F900F90DF91CF910895CF93B8
:102DD000DF93EC01EC81F0E0E65BFE4F4491E9E625
:102DE000F2E0628181810E94CC168C818F5F8C839E
:102DF000DF91CF910895CF93DF93EC01E9E6F2E004
:102E0000438162818C810E94CC168C818F5F8C8380
:102E1000DF91CF9108950F931F93CF93DF9300D04D
:102E200000D0CDB7DEB78C018091380281110AC085
:102E30009E012F5F3F4F4FEF6FEF0E94F6158A8183
:102E400080933802F8018481813051F028F082307B
:102E500061F4409138020AC08091380240E007C016
:102E60006091380240E080E003C040E080E060E034
:102E70000E94B316F801848190E0019663E070E04F
:102E80000E94C92884830F900F900F900F90DF91BC
:102E9000CF911F910F910895AF92BF92CF92DF9281
:102EA000EF92FF920F931F93CF93DF9300D000D048
:102EB000CDB7DEB7182FF62E042FE22E90916902BF
:102EC00090FF6CC0E92FE695AE2FB0E0AB56BE4F39
:102ED0008C91809342029E7F923061F49E012F5F1D
:102EE0003F4F812F0E94F6154B8169818A810E9494
:102EF000B31642C0823019F400916C023DC0863096
:102F000019F410916A0238C08930D9F38931A1F5DA
:102F1000E9518E2F8170D82EE695F0E0E65BFD4FEB
:102F2000A590B490C12CBB2460911301C61610F576
:102F30002C2D30E0A29EC001A39E900DB29E900D5C
:102F4000112470E00E94B528812FD11002C0860F95
:102F500001C0861B90911101290F311D220F331FD3
:102F6000220F331F22593D4F402F6F2D0E94F6151F
:102F7000C394DACF0E94761610936A02F0926B0225
:102F800000936C02EE2051F06091690270916A0228
:102F900080916B0290916C020E941C160F900F9012
:102FA0000F900F90DF91CF911F910F91FF90EF90B5
:102FB000DF90CF90BF90AF900895E9E6F2E0918165
:102FC000282F4381628188E0890F0C944C1781E09F
:102FD0000C94DD17E9E6F2E09181282F43816281AC
:102FE00088EF890F0C944C1781E00C94EA17E9E6FE
:102FF000F2E0628128E0620F08F46FEF282F43812E
:1030000081810C944C1781E00C94F717E9E6F2E00B
:10301000628128E0621B08F460E0282F43818181EF
:103020000C944C1781E00C940618E9E6F2E0438119
:1030300028E0420F08F44FEF282F628181810C9421
:103040004C1781E00C941518E9E6F2E0438128E082
:10305000421B08F440E0282F628181810C944C17B8
:1030600081E00C94241820E00C944C17FF920F93ED
:103070001F93CF93DF93EC01F12C0FEF10E06091E1
:103080001301F616E8F4809111012F2D30E0280F7E
:10309000311D220F331F220F331F22593D4F70E085
:1030A000C8010E94C928962F8C8140916C026091C2
:1030B0006B02F99E800D11240E94F615F394DFCF68
:1030C0000E9476169A818C8190FF02C08F5F01C0AA
:1030D00081508C83DF91CF911F910F91FF900895C4
:1030E000BF92CF92DF92EF92FF920F931F93CF93F5
:1030F000DF93FC01828180FF02C00FEF01C001E07D
:1031000010E080911301181708F040C08091110160
:10311000C12ED12CE601C80FD11DCC0FDD1FCC0F65
:10312000DD1FC259DD4F198218821A821B8224E0EA
:10313000E22EF12CB12C80913A028B0D823034F4C6
:1031400087FF05C090911301890F01C080E0082E10
:10315000000C990BC816D90691F480916C028E9DD3
:10316000A0018F9D500D1124559547955595479574
:103170009E0160916B0280916A020E94F615B00E6A
:10318000F1E0EF1AF108B9F61F5FBBCF0E94761687
:1031900080913A02013031F4811102C08091130113
:1031A000815007C090E001966091130170E00E9489
:1031B000C92880933A02DF91CF911F910F91FF9020
:1031C000EF90DF90CF90BF9008950F931F93CF9310
:1031D0008091110190911201891760F424E0829F7F
:1031E000F0011124E259FD4F1182108212821382E4
:1031F0008F5FF2CFC0E060911301C61798F50C2FD6
:1032000010E070E0C8010E94C928E09111018E0F02
:1032100020913902022E000C330BE82FF0E0EE0F64
:10322000FF1FEE0FFF1F02171307A4F080910E017E
:10323000082E000C990B8017910764F09F0122590A
:103240003D4F40916C0260916B0280916A020E9436
:10325000F61506C0E259FD4F1182108212821382C8
:10326000CF5FC9CF0E94761620910D01809139025F
:10327000820F8093390290910E01920F90930E016C
:1032800019165CF4082E000C990B4091130150E0C4
:1032900041505109841795071CF0219520930D0189
:1032A000CF911F910F9108958F929F92AF92BF92ED
:1032B000CF92DF92EF92FF920F931F93CF93DF9302
:1032C000EC014C81042F10E09801D8010E940D29D7
:1032D0009B01AC010E9423296B017C01E0E2F0E03C
:1032E000E01BF10BA5E5B0E09B01AC010E94232996
:1032F0004B015C019F01DF010E9405299B01AC018C
:103300000E942E299B01AC012C0D3D1D4E1D5F1D01
:10331000C501B4010E94DD28822F022F2A3228F431
:1033200093E0299F900111240DC025E530E0281B72
:103330003109C901880F991F280F391F37FF02C0B3
:103340002F5F3F4F35952795122F1095F12C85E56E
:10335000E82EE01A80911301F816C0F4F1FC02C0C7
:103360008E2D01C0802F909111012F2D30E0290F5B
:10337000311D220F331F220F331F22593D4F412F82
:1033800060916B020E94F615F394E4CF0E947616CA
:103390008C81811102C091E003C0803219F49FEF4B
:1033A00090930C0190910C01890F8C83DF91CF9148
:1033B0001F910F91FF90EF90DF90CF90BF90AF9053
:1033C0009F908F9008950F931F93CF93DF93EC01FD
:1033D00000E010E080911301282F30E0021713075E
:1033E0001CF5909111019801290F311D220F331FF7
:1033F000220F331F22593D4F869590E04C810817CC
:1034000019071CF4442331F002C0411103C040915C
:103410006C0201C040E060916B0280916A020E94E0
:10342000F6150F5F1F4FD6CF0E9476168C8190E065
:103430000196817099278C83DF91CF911F910F9115
:103440000895E9E6F2E080818E7F8083608171815A
:10345000828193810E941C16109243022FEF80E715
:1034600092E0215080409040E1F700C000000C94B1
:10347000761660916902669570E04BE050E084E159
:1034800091E00E943629892B19F481E08093430250
:103490000E948B2190933C0280933B02089590916F
:1034A000690290FF35C09170811102C0926006C020
:1034B000853210F0986402C0880F982B90936902AF
:1034C000662351F06091690270916A0280916B02EB
:1034D00090916C020E941C1660916902669570E0E2
:1034E0004BE050E084E191E00E943629892B19F0ED
:1034F0001092430202C00E94391A81E080933E027A
:1035000040916C0260916B0280916A020C943318B6
:103510000895682F90916902969581E0890F853210
:1035200008F081E00C944F1A81E00C94891A682FFE
:103530009091690296958FEF890F09F484E20C94BB
:103540004F1A81E00C94971A61E00C944F1AE9E647
:10355000F2E080818160808386950C94A41A80912A
:10356000690280FD0C94211A0C94A71A60E00C9457
:103570004F1A8091410281112EC00E94A90D811124
:1035800004C00E94510E0E942E160E9418166093CD
:10359000690270936A0280936B0290936C026E7F53
:1035A00061F40E942E160E941816609369027093AF
:1035B0006A0280936B0290936C020E94051610922F
:1035C00043028091690280FF03C086950E94B61A6B
:1035D00081E08093410208950F931F93CF93DF936F
:1035E00080914302882309F485C080914202E091D2
:1035F0006902E695E81BE0933D02823049F4F0E071
:10360000EA5BFE4FE491CE2FD0E007EE16E149C011
:10361000863049F4F0E0ED5BFE4FE491CE2FD0E030
:103620000BEF16E13EC0893051F4E695F0E0E05C26
:10363000FE4FE491CE2FD0E006E318E132C08F3088
:1036400051F4E695F0E0E35CFE4FE491CE2FD0E03C
:1036500000E718E126C0853149F4F0E0E65CFE4F52
:10366000E491CE2FD0E005EE18E11BC0883181F047
:10367000833239F4E8E3F1E0C591D4910BE017E12E
:1036800010C0843251F4C4EFD1E003EE19E109C057
:10369000C8E2D0E004E519E104C0C0EDD7E002EFD4
:1036A00015E180913E02882361F010923E020E9453
:1036B0008B2190933C0280933B0210924002109227
:1036C0003F020E948B21E0913B02F0913C028E1B55
:1036D0009F0B8F3F9F4770F4EC0FFD1FF0933C0250
:1036E000E0933B028BE392E0F801DF91CF911F91D1
:1036F0000F910994DF91CF911F910F910895882325
:1037000011F0FA0101C0FB010994CF93DF93C82F98
:10371000D62F0E943D168C1740F00E943D168D1743
:1037200020F4DF91CF910C94941A8C2FDF91CF91DC
:103730000C94A41A1F93CF93DF93FB0112811111F4
:10374000C3C0EC010E94C00C8272CD3CFCE5DF07D7
:1037500009F49AC0A8F5C73CECE5DE0709F476C089
:10376000A8F4C43C9CE5D90709F45FC028F4C33C25
:10377000DC4509F457C054C0C53C9CE5D90709F4A1
:1037800059C0C63CDC4509F45CC04AC0CA3CFCE5F3
:10379000DF0709F46AC050F4C83CECE5DE0709F421
:1037A0005AC0C93CDC4509F45BC03AC0CB3C9CE53F
:1037B000D90709F45FC0CC3CDC4509F460C030C0D7
:1037C000C23DFCE5DF0709F46FC088F4CF3C9CE5FF
:1037D000D90709F460C008F45CC0C03DFCE5DF0710
:1037E00009F45CC0C13DDC4509F45BC019C0C53DAE
:1037F0009CE5D90709F460C050F4C33DFCE5DF0740
:1038000009F455C0C43DDC4509F454C009C0C63DA7
:103810009CE5D90709F455C0CE35DD4509F454C0FF
:1038200011E052C00E94AF1A4FC041EA5AE164E968
:103830007AE104C044E95AE161EA7AE10E947F1B1F
:1038400043C044EF57E167EE77E1F8CF47EE57E129
:1038500064EF77E1F3CF42E158E163E078E1EECF46
:1038600043E058E162E178E1E9CF40E358E161E209
:1038700078E1E4CF41E258E160E378E1DFCF40E76F
:1038800056E169E576E1DACF49E556E160E776E1B0
:10389000D5CF81E017C065E082E010C068E086E027
:1038A0000DC06EE089E00AC064E18FE007C067E107
:1038B00085E104C088E106C062E289E10E94851BBF
:1038C00003C083E20E94A41A812FDF91CF911F9140
:1038D0000895519A2BB12D7F3BB132604FB7F894C8
:1038E000FC01660F771F660F771F6E0F7F1FE617AD
:1038F000F70789F0819198E03BB9000000C087FF8D
:103900002BB9880F000000C000C000C02BB900C058
:103910009A9591F7ECCF4FBF8FE594E00197F1F7BF
:1039200000C000000895CF93DF93EC01FB0182817A
:10393000882309F43CC1C430FDE5DF0760F4CB3FC8
:103940009CE5D90788F49E0122503C45243131057D
:1039500008F02EC109C0C236EDE5DE0729F0C63AEF
:10396000FDE5DF0709F024C10E94BC0D90936202BF
:1039700080936102C1318CE5D80709F4C6C008F014
:1039800042C0C930ECE5DE0709F49BC000F5C53044
:103990008CE5D80709F485C078F4C330ECE5DE0780
:1039A00009F478C008F07AC0C230DC4509F0F5C0EF
:1039B000809161028160EFC0C7309CE5D90709F4AE
:1039C00078C008F07AC0809161028061E4C0CD3097
:1039D000FCE5DF0709F487C058F4CB309CE5D90734
:1039E00009F479C008F07BC08091610288606FC0E3
:1039F000CF30FCE5DF0709F480C008F082C0809179
:103A00006102877FC8C0CE3F9CE5D90709F471C029
:103A100000F5C531FCE5DF0709F485C068F4C33162
:103A20009CE5D90709F475C008F095C00E946F079E
:103A3000809161028F77AFC0CC3FFCE5DF07A9F131
:103A400008F054C0CB3FDC4509F0A7C0809162026A
:103A500040C0C230EDE5DE0709F489C058F4C11555
:103A60008DE5D80709F45AC008F069C08091620258
:103A700082602FC0C236EDE5DE0709F47CC0C63A8D
:103A8000FDE5DF0709F481C0C330DD4509F085C0DD
:103A900080E06EC08091610282607DC08091610291
:103AA00016C080916102886076C080916202826057
:103AB0004FC08091610280626EC08091610280641B
:103AC0006AC00E946F0780916102806864C0846050
:103AD00062C081603DC0809161028E7F5CC0809138
:103AE00061028D7F58C08091610216C08091620290
:103AF00018C0809162028D7F2BC0809161028F7E01
:103B00004AC0809161028F7D46C0809161028F7BA7
:103B100042C080916102877F8B7F3DC080916202AD
:103B20008D7F8E7F15C08091610282FB222720F954
:103B300091E0922790FB82F990FB83F92CC0809151
:103B40006202982F909591708E7F892B90FB81F95E
:103B50008093620222C00E946F078091610287FBFE
:103B6000222720F991E0922790FB87F914C081E089
:103B70000E94530E12C08091610284FB222720F91B
:103B800091E0922790FB84F906C080916102982F02
:103B9000909590FB80F980936102809161029091F1
:103BA00062020E94CD0D0E946F0780E001C081E09B
:103BB000DF91CF910895893289F1F0F4843171F168
:103BC000B0F4873009F077C081E080930B0184E185
:103BD00080930A018AE0809309018EE180930801B5
:103BE00088E08093050188E28093040164C092EE2E
:103BF000980F9A30F0F05FC0803509F444C028F483
:103C00008F3409F058C08AE03FC0813529F08235F1
:103C100009F051C081E038C08FEF36C08091460274
:103C2000882379F1109246021092450210924402C4
:103C300042C08D5180934602833099F038F4813030
:103C400069F08230D9F48AE091E00DC0853099F0B6
:103C500078F0863099F484E091E005C08BE091E043
:103C600002C089E091E0909345028093440223C012
:103C700088E091E0F8CF85E091E0F5CF1092460220
:103C80001AC080E0089586EFE0914402F091450269
:103C9000309789F02081082E000C990B820F911D1E
:103CA0008F3F910519F014F08FEF04C097FF02C009
:103CB000108201C0808381E008950F931F9341E03B
:103CC00050E060E070E08A019B0104C0000F111F0A
:103CD000221F331F8A95D2F7C901B8010E94C70776
:103CE0001F910F910C946F078B3109F468C058F540
:103CF0008B3009F486C078F4863009F445C020F48E
:103D0000853009F44BC07FC0873009F44AC0883041
:103D100009F477C078C0803109F464C068F48E304B
:103D200009F071C08091270282FB222720F991E0DF
:103D3000922790FB82F94CC0863109F462C0893128
:103D400009F45FC060C08A32E1F060F4873209F4A0
:103D500055C028F48E3108F456C08D5150C08932B8
:103D6000E9F051C0833450F48A3308F045C08533FC
:103D700009F444C0883309F444C045C08334F1F1E8
:103D800042C00E94510E3DC080912702817F8E7FEC
:103D90008093270281E08093470208950E94B20237
:103DA00030C080912702982F9095917090FB80F9F8
:103DB00080932702911125C0897F877F10C0809151
:103DC000270281FB222720F991E0922790FB81F9BD
:103DD000809327029923A9F0809127028160809324
:103DE00027020FC08091270283FB222720F991E050
:103DF000922790FB83F9ECCF895301C080E00E94A9
:103E00005D1E81E0089580E0089580E008950C949F
:103E1000051FCF93C82F80914702813069F038F099
:103E20008230C1F58C2F0E94DB1D81E039C00E94D9
:103E3000C00C823289F504C00E94C00C823261F449
:103E40008C2F0E94071F811104C08C2F0E94741EAA
:103E50001FC081E090E01CC08C2F0E94051F8111C3
:103E600016C0C43189F058F4CB3089F0C031B1F4B8
:103E700082E08093470288E30E94DB1D08C0C932BC
:103E800019F0C83321F00AC01092470207C081E040
:103E9000817006C01092470280E002C080E0F8CF37
:103EA000CF910895CF93DF9386319C4541F5EB0187
:103EB0000E94C00C982F8A81209102013091030149
:103EC000882379F09A7A81E009F480E080934802AF
:103ED000911102C069E201C065E3C9010E94E520B9
:103EE0000AC080914802811102C069E201C065E305
:103EF000C9010E94E7200E94020D80E001C081E01C
:103F0000DF91CF9108950F931F93CF93DF93C42F29
:103F1000D22FFC0182818823C9F040934B020E947A
:103F20008B2190934A028093490280E28C0F883063
:103F300008F057C0C77081E001C0880FCA95EAF742
:103F4000DF91CF911F910F910C94CC0480914B0283
:103F5000481330C08091490290914A020E94A321E7
:103F6000883C910538F510E21D0FCD17B9F080E2BD
:103F70008C0F883040F4C77081E001C0880FCA956B
:103F8000EAF70E94D304183028F581E09D2F97703E
:103F900001C0880F9A95EAF70E94CC04802F0E94F6
:103FA000C3041830F0F4D77081E001C0880FDA95AF
:103FB000EAF70AC080E28C0F883098F4C77081E07D
:103FC00001C0880FCA95EAF7DF91CF911F910F9139
:103FD0000C94D304802FDF91CF911F910F910C94FB
:103FE000C304DF91CF911F910F9108950F939C010E
:103FF000CB01243F4CE5340731F188F4293DFCE541
:104000003F07D9F02A3D4CE5340779F1283D3C457E
:10401000A9F506E221EE41EE68ED7CE52BC0263FD6
:10402000FCE53F07E1F0A8F0273F3C4539F507E202
:1040300025EE46EE67EF7CE51DC007E225EE45EE76
:1040400069ED7CE517C006E221EE40EE64EF7CE509
:1040500011C007E225EE44EE65EF7CE50BC006E2F9
:1040600021EE42EE66EF7CE505C008E221E045EE78
:104070006AED7CE50E94831F80E008C0FC0182811C
:10408000882319F010924B0201C081E00F9108952E
:104090009093BB018093BA0108959093510280934D
:1040A00050020895E0915002F0915102309721F0B2
:1040B0000190F081E02D099480E00895E091500294
:1040C000F0915102309721F00280F381E02D0994A4
:1040D0000895E0915002F0915102309739F022E0BA
:1040E000DC012C930480F581E02D09940895209142
:1040F0004E0230914F022817390771F090934F020A
:1041000080934E02E0915002F0915102309721F0DD
:104110000680F781E02D0994089520914C0230919A
:104120004D022817390771F090934D0280934C028D
:10413000E0915002F0915102309721F00084F18516
:10414000E02D09940895FC01329697E080E09150AB
:1041500029F021912223D9F38F5FF9CF08956623A7
:1041600049F0FC01329608962191621729F0E81770
:10417000F907D1F780E0089581E008959C01FC01E2
:1041800032969FEF80E04191461789F09F3F19F4E6
:10419000411101C0982F8F5F8630A9F79F3F39F0FA
:1041A000F901E90FF11D97FDFA95628308950895CD
:1041B0009C012A5F3F4FFC014281461301C01282DD
:1041C000019682179307B9F708950C94BE200C94BA
:1041D000D820029626E0FC0111922A95E9F708956D
:1041E00008950C94F02083E0809352020C94F12007
:1041F000811102C081E001C082E0809352020C94E0
:10420000F1200C94F82081E0809352020C94F1206C
:104210000C94032108950C940A210C940B210C9406
:104220000A210C940A210C940A21CF930E94112197
:104230000E942F120E940F21C0E08C2F0E946E114D
:10424000811104C0CF5FC330C1F701C081E0CF91BD
:10425000089508951F920F920FB60F9211248F9315
:104260009F93AF93BF9380915302811113C08091AC
:10427000720290917302A0917402B09175024196FE
:10428000A11DB11D8093720290937302A0937402DA
:10429000B0937502BF91AF919F918F910F900FBE18
:1042A0000F901F90189580917A02843031F10E940E
:1042B0001A031092530220E488E190E00FB6F894BC
:1042C000A895809360000FBE2093600083B7817F24
:1042D000846083BF83B7816083BF7894889583B7F8
:1042E0008E7F83BF0FB6F894A89580916000886197
:1042F00080936000109260000FBE08950E946F07C7
:104300000C941E0382E084BD93E095BD9AEF97BDA7
:1043100080936E0008952FB7F89480917202909167
:104320007302A0917402B09175022FBF08952FB748
:10433000F89460917202709173028091740290916E
:1043400075022FBF08959C014FB7F89480917202B7
:1043500090917302A0917402B09175024FBF821BBD
:10436000930B089578941F920F920FB60F92112419
:104370008F939F93AF93BF9380917202909173023A
:10438000A0917402B09175020196A11DB11D809398
:10439000720290937302A0937402B0937502BF915E
:1043A000AF919F918F910F900FBE0F901F90189516
:1043B00087E797E790930108809300089AE088E1E7
:1043C0000FB6F894A895809360000FBE909360009C
:1043D000FFCF80915F020895089522E02093E900C5
:1043E0002FEF3091E800215035FD06C035ED3A95AC
:1043F000F1F700002111F5CF2091E80025FF0BC057
:1044000040E050E066E070E00E9417248091E800F0
:104410008E778093E8000895CF93DF9321E0209377
:10442000E9002FEF3091E800215035FD06C035ED51
:104430003A95F1F700002111F5CF2091E80025FF12
:1044400014C0EC0140E050E068E070E00E941724E6
:104450008091E8008E778093E80088E0FE01A7E570
:10446000B2E001900D928A95E1F7DF91CF91089526
:1044700080935402709356026093550280917A02A1
:10448000843001F582E08093E9008FEF9091E8009D
:10449000815095FD06C095ED9A95F1F700008111C8
:1044A000F5CF8091E80085FF0DC040E050E063E06B
:1044B00070E084E592E00E9417248091E8008E77F6
:1044C0008093E8000895BC0184E00C943822BC017C
:1044D00083E00C94382280917902811109C00E94F6
:1044E000A8250E9405268091E20084608093E20066
:1044F00008951092790208950C9408216091760233
:1045000081E0611101C080E00C94F32090917A0267
:1045100081E0943009F080E0609176020C94F820FC
:1045200042E061EC81E00E94212542E261EC82E000
:104530000E94212590917A0281E0943009F080E078
:10454000609176020C94012180917C02833009F401
:1045500061C030F4813071F0823009F49AC008955E
:104560008A3009F486C08B3009F46CC0893009F0B8
:10457000A8C020C080917B02813A09F0A2C080913E
:10458000E800877F8093E80080917F02909180020D
:10459000892B21F468E087E592E003C060E080E0C9
:1045A00090E070E00E9462248091E8008B77809315
:1045B000E800089580917B02813209F082C08091E9
:1045C0007F0290918002029708F07BC08091E80002
:1045D000877F8093E8008091E80082FD05C080918C
:1045E0007A028111F8CF6DC02091F3008091F20022
:1045F00090E0922B029731F48091F100813011F01C
:10460000863021F48091F10080935F028091E80070
:104610008B7753C080917B02813A09F052C0809120
:104620007F0290918002892B09F04BC08091E800B5
:10463000877F8093E8008091E80080FFFCCF809125
:104640002B0136C080917B028132D9F580917F02A7
:1046500090918002892BA9F58091E800877F809353
:10466000E8000E94562580917D0280932B010C94D6
:104670006F0780917B02813221F58091E800877F6E
:104680008093E8000E94562580917E02809360020C
:10469000089580917B02813AA1F48091E800877FA0
:1046A0008093E8008091E80080FFFCCF8091600259
:1046B0008093F1008091E8008E778093E8000C945D
:1046C0005625089584B7877F84BF0FB6F894A895C0
:1046D00080916000886180936000109260000FBE3E
:1046E00090E080E80FB6F8948093610090936100A9
:1046F0000FBE0C9403210E94A8250E940526E2EE1D
:10470000F0E080818460808378940C949A288FE113
:1047100091E00C944D2080917A028530A9F480912B
:104720007A02853079F40E9453218091780288239F
:10473000B1F30E941521882391F30E9401240E9465
:104740006F07EDCF0C947E21089508950C94A82353
:10475000292F332723303105C9F060F4213031058A
:1047600081F02230310509F044C08BE390E02FE660
:1047700033E043C021323105E1F02232310549F105
:1047800038C082E190E02AEA33E037C099278130CF
:10479000910549F028F0029761F5EFE4F3E005C0D8
:1047A000EBE6F3E002C0EFE5F3E0849190E09F01D7
:1047B00024C06115710541F061307105D1F489E0C3
:1047C00090E02AE933E019C089E090E021E833E085
:1047D00014C06115710541F06130710551F48BE72A
:1047E00090E02CEB33E009C080E490E027E334E074
:1047F00004C080E090E020E030E0FA0131832083C3
:10480000089580E189BD82E189BD09B400FEFDCF34
:104810008091D8008F7D8093D8008091E0008260E5
:104820008093E0008091E00081FDFCCF0895CF925D
:10483000DF92EF92FF920F931F93CF93DF93EC01E0
:104840008B017A010E947525811133C0E114F104B6
:1048500039F0F70180819181081B190BC80FD91F0E
:10486000C12CD12C0115110519F18091E80085FDAD
:1048700016C08091E8008E778093E800E114F1047F
:1048800049F0F70180819181C80ED91ED182C08282
:1048900085E00FC00E947525882321F30AC0899105
:1048A0008093F10001501109FFEFCF1ADF0ADACF30
:1048B00080E0DF91CF911F910F91FF90EF90DF90FB
:1048C000CF900895209181023091820226173707F8
:1048D00048F06115710539F42091E8002E77209396
:1048E000E80001C0B901FC0120E06115710579F112
:1048F00080917A028823F1F18530F1F18091E8000E
:1049000083FD3CC08091E80082FD2EC08091E800CC
:1049100080FFEBCF2091F3008091F20090E0922B8A
:104920006115710551F08830910538F4219120937B
:10493000F100615071090196F3CF21E0089709F069
:1049400020E08091E8008E778093E800CECF21119F
:10495000CFCF0AC080917A02882361F0853061F060
:104960008091E80083FD0AC08091E80082FFF2CFC9
:1049700080E0089582E0089583E0089581E008953D
:1049800020918102309182022617370748F0611585
:10499000710539F42091E8002E772093E80001C0DA
:1049A000B901FC0120E06115710591F180917A0255
:1049B000882309F440C0853009F43FC08091E800A5
:1049C00083FD3DC08091E80082FD2FC08091E8000A
:1049D00080FFE9CF2091F3008091F20090E0922BCC
:1049E0006115710559F08830910540F424912093A8
:1049F000F1003196615071090196F2CF21E00897DC
:104A000009F020E08091E8008E778093E800CBCF1A
:104A10002111CCCF0AC080917A02882361F08530C1
:104A200061F08091E80083FD0AC08091E80082FF78
:104A3000F2CF80E0089582E0089583E0089581E058
:104A40000895982F973068F59093E900981739F0FA
:104A50007091EC002091ED005091F00003C0242FE4
:104A6000762F50E021FD02C09F5FECCF3091EB002C
:104A70003E7F3093EB003091ED003D7F3093ED00B1
:104A80003091EB0031603093EB007093EC00209399
:104A9000ED005093F0002091EE0027FDE5CF80E07F
:104AA00008958F708093E90081E0089580917B02E2
:104AB00087FF11C08091E80082FD05C080917A02D5
:104AC0008111F8CF11C08091E8008B770BC08091E5
:104AD0007A02882349F08091E80080FFF8CF809126
:104AE000E8008E778093E80008952091E4003091EB
:104AF000E50095E64091EC00842F817040FF23C0D3
:104B00008091E80080FD1DC080917A02882399F091
:104B1000853099F08091EB0085FD11C04091E40053
:104B20005091E5002417350729F3915011F09A01AF
:104B3000E1CF84E0089582E0089583E0089581E064
:104B4000089580E008954091E80042FFDDCF089588
:104B50000E9416260E941E26E0EEF0E08081816011
:104B60008083E8EDF0E080818F77808319BCA7ED2A
:104B7000B0E08C918E7F8C9380818F7E80831092A9
:104B8000790208950F931F93CF93DF930E94162607
:104B90000E941E26C8EDD0E088818F7788838881A7
:104BA0008068888388818F7D888319BC10927A02FF
:104BB00010927602109278021092770200EE10E0C6
:104BC000F80180818B7F808388818160888342E0C7
:104BD00060E080E00E942125E1EEF0E080818E7FA0
:104BE0008083E2EEF0E08081816080838081886054
:104BF0008083F80180818E7F8083888180618883B3
:104C0000DF91CF911F910F910895E8EDF0E0808141
:104C10008F7E8083E7EDF0E080818160808384E097
:104C200082BF81E0809379020C94C225E8EDF0E028
:104C300080818E7F80831092E20008951092DA00C6
:104C40001092E10008951F920F920FB60F92112457
:104C50002F933F934F935F936F937F938F939F9384
:104C6000AF93BF93EF93FF938091E10082FF0BC05E
:104C70008091E20082FF07C08091E1008B7F8093EA
:104C8000E1000E9499288091DA0080FF1FC0809186
:104C9000D80080FF1BC08091DA008E7F8093DA00FD
:104CA0008091D90080FF0DC080E189BD82E189BD7E
:104CB00009B400FEFDCF81E080937A020E946B224E
:104CC00005C019BC10927A020E9479228091E100FD
:104CD00080FF19C08091E20080FF15C08091E20042
:104CE0008E7F8093E2008091E20080618093E200F9
:104CF0008091D80080628093D80019BC85E08093B1
:104D00007A020E947E228091E10084FF30C080916F
:104D1000E20084FF2CC080E189BD82E189BD09B435
:104D200000FEFDCF8091D8008F7D8093D8008091C8
:104D3000E1008F7E8093E1008091E2008F7E80937E
:104D4000E2008091E20081608093E200809176022F
:104D5000882311F084E007C08091E30087FD02C042
:104D600081E001C083E080937A020E9486228091D4
:104D7000E10083FF29C08091E20083FF25C080917C
:104D8000E100877F8093E10082E080937A021092B5
:104D900076028091E1008E7F8093E1008091E200B5
:104DA0008E7F8093E2008091E20080618093E20038
:104DB00042E060E080E00E9421258091F000886060
:104DC0008093F0000E947C22FF91EF91BF91AF9100
:104DD0009F918F917F916F915F914F913F912F9113
:104DE0000F900FBE0F901F9018951F920F920FB645
:104DF0000F9211242F933F934F935F936F937F9361
:104E00008F939F93AF93BF93CF93DF93EF93FF93D2
:104E1000C091E900CF708091EC00D82FD17080FD57
:104E2000D0E81092E9008091F000877F8093F00035
:104E300078940E9439271092E9008091F0008860F0
:104E40008093F000CD2BCF70C093E900FF91EF91DC
:104E5000DF91CF91BF91AF919F918F917F916F9192
:104E60005F914F913F912F910F900FBE0F901F9028
:104E700018951F93CF93DF93CDB7DEB7AA970FB6E0
:104E8000F894DEBF0FBECDBFEBE7F2E08091F100FA
:104E9000819322E0E338F207C9F70E94A4228091AF
:104EA000E80083FF2EC180917B0290917C02492F04
:104EB00050E04A30510508F024C1FA01EE59FF4F85
:104EC0000C94FF28803821F0823809F01AC108C0FC
:104ED0008091770290917802992389F082600FC0C7
:104EE00080917F028F70873008F00BC18093E900BA
:104EF0008091EB0085FB882780F91092E900909162
:104F0000E800977F9093E8008093F1001092F10001
:104F1000D1C0282F2D7F09F0F4C0882319F08230EA
:104F200061F0EFC080917D02813009F0EAC09330DA
:104F300009F080E0809378022EC080917D0281117B
:104F40002AC080917F028F702FEF280F263008F043
:104F5000D8C08093E9002091EB0020FF1CC0933063
:104F600021F48091EB00806214C09091EB0090617D
:104F70009093EB0021E030E0A90102C0440F551FDF
:104F80008A95E2F74093EA001092EA008091EB00E4
:104F900088608093EB001092E9008091E800877FA1
:104FA0008093E8000E945625ACC08111AAC01091E0
:104FB0007D021F778091E3008078812B8093E3004E
:104FC0008091E800877F8093E8000E9456258091B9
:104FD000E80080FFFCCF8091E30080688093E300CD
:104FE000111102C082E001C083E080937A0289C07F
:104FF0008058823008F085C080917D0290917E02B9
:105000008C3D53E0950779F583E08A838AE28983B2
:105010004FB7F894DE01139620E03EE051E2E32F13
:10502000F0E050935700E49120FF03C0E295EF7049
:105030003F5FEF708E2F90E0EA3010F0C79601C00E
:10504000C0968D939D932F5F243149F74FBF809178
:10505000E800877F8093E8006AE270E0CE01019665
:105060000E94622416C060917F0270918002AE019E
:105070004F5F5F4F0E94A623BC01892B09F441C0FA
:105080009091E800977F9093E80089819A810E942F
:10509000C0248091E8008B778093E80032C080388C
:1050A00081F58091E800877F8093E8008091760207
:1050B0008093F1008091E8008E7772CF811121C03A
:1050C00080917D0290917E0299270297D4F480917D
:1050D000E800877F8093E80080917D0280937602CC
:1050E0000E94562580917602811106C08091E300CE
:1050F00087FD02C081E001C084E080937A020E94B3
:1051000090228091E80083FF0AC08091E800877FA9
:105110008093E8008091EB0080628093EB00AA9678
:105120000FB6F894DEBF0FBECDBFDF91CF911F91B8
:1051300008950895CF9380917A028823A1F0C091B9
:10514000E900CF709091EC00892F817090FD80E88C
:10515000C82B1092E9008091E80083FD0E94392756
:10516000CF70C093E900CF910895AA1BBB1B51E1FA
:1051700007C0AA1FBB1FA617B70710F0A61BB70BC7
:10518000881F991F5A95A9F780959095BC01CD016C
:10519000089597FB072E16F4009407D077FD09D0E9
:1051A0000E94B52807FC05D03EF4909581959F4F4D
:1051B0000895709561957F4F0895A1E21A2EAA1B5C
:1051C000BB1BFD010DC0AA1FBB1FEE1FFF1FA217B7
:1051D000B307E407F50720F0A21BB30BE40BF50BB4
:1051E000661F771F881F991F1A9469F7609570953D
:1051F000809590959B01AC01BD01CF010895EE0F04
:10520000FF1F0590F491E02D09940E940D2933238E
:1052100012F48A1B9B0B0C941E29A29FB001B39F12
:10522000C001A39F700D811D1124911DB29F700DAF
:10523000811D1124911D08950E940D29B7FF089525
:10524000821B930B08950E940D29A59F900DB49F7A
:10525000900DA49F800D911D11240895B7FF0C940B
:1052600023290E942329821B930B0895FC0141509E
:10527000504030F001900616D1F73197CF010895D4
:10528000882799270895FB01DC0104C08D910190C6
:10529000801921F441505040C8F7881B990B08959C
:1052A000F999FECF92BD81BDF89A992780B50895EE
:1052B000A6E1B0E044E050E00C948A29A8E1B0E017
:1052C00042E050E00C948A29262FF999FECF92BD36
:1052D00081BDF89A019700B4021639F01FBA20BDBB
:1052E0000FB6F894FA9AF99A0FBE08950396272FED
:1052F0000E9465290E946429252F0E946529242F78
:105300000C9465290196272F0E9465290C94642925
:10531000DC01CB01FC01F999FECF06C0F2BDE1BD75
:10532000F89A319600B40D9241505040B8F7089564
:04533000F894FFCF1F
:10533400C8001202280850011E0A140101010200CB
:105344000100010101191A1B1C1D1E1F202122E945
:10535400210C22ED2167226322EC2101E200E90005
:10536400EA00B500B600B700CD008301CC008A0185
:10537400920194012102230224022502260227021B
:105384002A02B300B4006F007000818283E200E956
:1053940000EA00B500B600B700CD008301CC008A56
:1053A40001920194012102230224022502260227EC
:1053B400022A02B300B4006F00700081828397C692
:1053C40034356694900001020202020606060909B9
:1053D400090909090F0F0F0F0F0F151515181919C2
:0A53E40019191919191919192324B0
:00000001FF
